:020000040000FA
:04000000FA3060284A
:080008008612601C8616AE0092
:10001000030EAF008312051E13284008E000601C89
:10002000861660188612051D1728BC0B1328283069
:10003000BC000F30A3008B100314851E0310E00CCE
:0A0040002F0E8300AE0E2E0E0900F5
:1000C000203084008001840A80300402031C6228EE
:1000D0002830BC008316FF3085055F308605FF3071
:1000E00087058312850186018701103083168E00F3
:1000F0008312703083168F0083120030031799002B
:100100000313003003179A000313003097000030E8
:100110009F00003083169F008312003003179E005B
:100120000313003003179F000313C73083168100A9
:10013000831230309000003092000030831694001B
:10014000831200309400A63083169800831200308A
:1001500083169B0083120030980033308316990079
:100160008312003083168C008312003083168D00BA
:10017000831210308B00B20BBB280130A400810128
:100180008E018F010B118B100B108C128C018D01C5
:100190008B1764000B19D920E820C92848085002A1
:1001A000031DD6285008871E5009C0004808D000FB
:1001B00008000B11A40B08000430A400A3080319C5
:1001C000E4288613A3030800060980398600080086
:1001D0000608A0000708A1002118F5280130871F94
:1001E0006430A5070318FC2803290130871F6430F9
:1001F000A502031C00290329FF30A5004814032988
:10020000A50148100329A1180C290130871F64306B
:10021000A607031813291A290130871F6430A60284
:10022000031C17291A29FF30A600C8141A29A60191
:10023000C8101A29211923290130871F6430A70704
:1002400003182A2931290130871F6430A702031CB3
:100250002E293129FF30A70048153129A70148115F
:100260003129201A3A290130871F6430A807031862
:10027000412948290130871F6430A802031C452901
:100280004829FF30A800C8154829A801C8114829E5
:10029000211A51290130871F6430AA0703185829F1
:1002A0005F290130871F6430AA02031C5C295F2983
:1002B000FF30AA0048165F29AA0148125F29201BB7
:1002C00068290130871F6430AB0703186F2976292E
:1002D0000130871F6430AB02031C73297629FF307D
:1002E000AB00C8167629AB01C8127629211B7F29DD
:1002F0000130871F6430AC07031886298D2901302F
:10030000871F6430AC02031C8A298D29FF30AC00A2
:1003100048178D29AC0148138D29A1199629013060
:10032000871F6430AD0703189D29A4290130871F5A
:100330006430AD02031CA129A429FF30AD00C81709
:0C034000A429AD01C813A429CE20080098
:084000000800000000000800A8
:02400E00CC03E1
:00000001FF
